:020000040000FA
:1000000019EF2AF0C96E120006EF13F0ACA2FED76A
:10001000AD6E1200C282120054EF25F0D350FC0BDB
:10002000D36ED3508F0B7009D36E0501416B426BB9
:100030000501436B446B0501456B466B30EC27F0C3
:100040008188000EE56E640EE56EB6EC25F0E65292
:10005000E6528198D6EC1BF0C9EC26F0006EF3CF87
:1000600001F00050400A03E10150120A01E01DD0E6
:10007000000E046E2F0E036E0A0E026E000E066E48
:10008000600E056E800E076E0450E56E0350E56E3F
:100090000250E56E0750E56E0650E56E0550E56EC0
:1000A00018EC23F0060EE12644D00050400A03E18C
:1000B00001502A0A01E01DD0000E046E2F0E036EBF
:1000C000220E026E000E066E600E056E800E076E2A
:1000D0000450E56E0350E56E0250E56E0750E56E84
:1000E0000650E56E0550E56E18EC23F0060EE1268D
:1000F00020D0000E046E2F0E036E3A0E026E000E1C
:10010000066E600E056E800E076E0150E56E0050A3
:10011000E56E0450E56E0350E56E0250E56E075043
:10012000E56E0650E56E0550E56E18EC23F0080EFE
:10013000E126000E016E600E006E800E026E02500F
:10014000E56E0150E56E0050E56E8DEC26F0030E75
:10015000E12602EC27F0050E016E500E006E800EB7
:10016000026E0250E56E0150E56E0050E56EA1ECA6
:1001700020F0006E030EE1260050EDE0FB0E0501BD
:10018000505DD8A067EF07F0050E5025006EFA6AA3
:10019000FB6A0034FA36E834FA36FC0BAC0FE56E35
:1001A000010EFA22000EFB22E450F96E61EF07F017
:1001B00030EF05F0FEEF02F0E0EF00F0F9EF01F0B4
:1001C00005EC2AF0000E026E2F0E016E660E006E18
:1001D0000250E56E0150E56E0050E56E8DEC26F0A4
:1001E000030EE126F9EC27F0006A016A270EE56E9E
:1001F000100EE56EB6EC25F0E652E65234EC28F02F
:10020000026EF3CF03F00350015C02E10250005C88
:1002100012E202C000F003C001F0000EE56EC80E4D
:10022000E56EB6EC25F0E652E65234EC28F0026EAC
:10023000F3CF03F0E8D70FEC2AF0000E066E2F0E76
:10024000056E800E046E000E086E600E076E800E46
:10025000096E0650E56E0550E56E0450E56E0950D6
:10026000E56E0850E56E0750E56E18EC23F0060EBB
:10027000E126000E056E600E046E800E066E0650BE
:10028000E56E0550E56E0450E56E8DEC26F0030E2C
:10029000E126046A056A34EC28F0066EF3CF07F015
:1002A0000750055C02E10650045CD8B04CD0050E46
:1002B000076E510E066E800E086E0850E56E0750F0
:1002C000E56E0650E56EA1EC20F0030EE12651C567
:1002D00006F0076A000E0A6E2F0E096E840E086E75
:1002E000000E0C6E600E0B6E800E0D6E0750E56EEC
:1002F0000650E56E0A50E56E0950E56E0850E56E51
:100300000D50E56E0C50E56E0B50E56E18EC23F0C9
:10031000080EE126000E076E600E066E800E086E57
:100320000850E56E0750E56E0650E56E8DEC26F040
:10033000030EE12605015151E56EFDEC21F0E65278
:10034000044A052AA8D7000E066E2F0E056E880EE9
:10035000046E000E086E600E076E800E096E065069
:10036000E56E0550E56E0450E56E0950E56E0850E7
:10037000E56E0750E56E18EC23F0060EE126000E40
:10038000056E600E046E800E066E0650E56E05501A
:10039000E56E0450E56E8DEC26F0030EE1266BEC65
:1003A00028F0050E056E500E046E800E066E065087
:1003B000E56E0550E56E0450E56EA1EC20F0046E8C
:1003C000030EE12604500FE005015051E56EFCECF0
:1003D00028F0E652000EE56E040EE56EB6EC25F050
:1003E000E652E652DED7C3EC29F002EC27F067EFC5
:1003F00007F0006A016A030EE56EE80EE56EB6ECE2
:1004000025F0E652E65234EC28F0026EF3CF03F00A
:100410000350015C02E10250005C12E202C000F0F5
:1004200003C001F0010EE56EF40EE56EB6EC25F0AA
:10043000E652E65234EC28F0026EF3CF03F0E8D730
:1004400005EC2AF0000E066E2F0E056E8C0E046E63
:10045000000E086E600E076E800E096E0650E56E87
:100460000550E56E0450E56E0950E56E0850E56EE6
:100470000750E56E18EC23F0060EE126000E056E1F
:10048000600E046E800E066E0650E56E0550E56E39
:100490000450E56E8DEC26F0030EE126046A056A31
:1004A00034EC28F0066EF3CF07F00750055C02E14C
:1004B0000650045CD8B04CD0050E076E510E066E87
:1004C000800E086E0850E56E0750E56E0650E56E2A
:1004D000A1EC20F0030EE12651C506F0076A000EDC
:1004E0000A6E2F0E096E840E086E000E0C6E600EE2
:1004F0000B6E800E0D6E0750E56E0650E56E0A50CD
:10050000E56E0950E56E0850E56E0D50E56E0C5035
:10051000E56E0B50E56E18EC23F0080EE126000E98
:10052000076E600E066E800E086E0850E56E07506E
:10053000E56E0650E56E8DEC26F0030EE126050112
:100540005151E56EFDEC21F0E652044A052AA8D788
:10055000000E066E2F0E056E880E046E000E086EDD
:10056000600E076E800E096E0650E56E0550E56E52
:100570000450E56E0950E56E0850E56E0750E56ED3
:1005800018EC23F0060EE126000E056E600E046ED8
:10059000800E066E0650E56E0550E56E0450E56E61
:1005A0008DEC26F0030EE1266BEC28F0050E056EAF
:1005B000510E046E800E066E0650E56E0550E56E17
:1005C0000450E56EA1EC20F0046E030EE126045009
:1005D0000FE005015151E56EFCEC28F0E652000EEB
:1005E000E56E040EE56EB6EC25F0E652E652DED777
:1005F000C3EC29F002EC27F067EF07F005EC2AF0D6
:1006000002EC27F0006A016A010EE56E900EE56EBD
:10061000B6EC25F0E652E65234EC28F0026EF3CF49
:1006200003F00350015C02E10250005C12E202C0E0
:1006300000F003C001F0000EE56EC80EE56EB6ECEA
:1006400025F0E652E65234EC28F0026EF3CF03F0C8
:10065000E8D705EC2AF0000E066E2F0E056E8C0E04
:10066000046E000E086E600E076E800E096E065056
:10067000E56E0550E56E0450E56E0950E56E0850D4
:10068000E56E0750E56E18EC23F0060EE126000E2D
:10069000056E600E046E800E066E0650E56E055007
:1006A000E56E0450E56E8DEC26F0030EE126046A3B
:1006B000056A34EC28F0066EF3CF07F00750055CAE
:1006C00002E10650045CD8B04CD0050E076E510E06
:1006D000066E800E086E0850E56E0750E56E0650F7
:1006E000E56EA1EC20F0030EE12651C506F0076A85
:1006F000000E0A6E2F0E096E840E086E000E0C6E30
:10070000600E0B6E800E0D6E0750E56E0650E56EA6
:100710000A50E56E0950E56E0850E56E0D50E56E25
:100720000C50E56E0B50E56E18EC23F0080EE12638
:10073000000E076E600E066E800E086E0850E56EA5
:100740000750E56E0650E56E8DEC26F0030EE126AF
:1007500005015151E56EFDEC21F0E652044A052AEF
:10076000A8D7000E066E2F0E056E880E046E000EC2
:10077000086E600E076E800E096E0650E56E05501D
:10078000E56E0450E56E0950E56E0850E56E0750C1
:10079000E56E18EC23F0060EE126000E056E600EE5
:1007A000046E800E066E0650E56E0550E56E045030
:1007B000E56E8DEC26F0030EE126F90EE56EAE0E29
:1007C000E56EDAEC27F0E652E652050E056E510EA4
:1007D000046E800E066E0650E56E0550E56E045000
:1007E000E56EA1EC20F0046E030EE12604500FE04C
:1007F00005015151E56E9DEC28F0E652000EE56EC4
:100800000C0EE56EB6EC25F0E652E652DED7EFECC4
:1008100029F0F90EE56EAE0EE56E7BEC27F0E652A0
:10082000E652006A016A010EE56E900EE56EB6ECC6
:1008300025F0E652E65234EC28F0026EF3CF03F0D6
:100840000350015C02E10250005C12E202C000F0C1
:1008500003C001F0000EE56EC80EE56EB6EC25F0A3
:10086000E652E65234EC28F0026EF3CF03F0E8D7FC
:10087000E4EC29F0000E066E2F0E056E800E046E5D
:10088000000E086E600E076E800E096E0650E56E53
:100890000550E56E0450E56E0950E56E0850E56EB2
:1008A0000750E56E18EC23F0060EE126000E056EEB
:1008B000600E046E800E066E0650E56E0550E56E05
:1008C0000450E56E8DEC26F0030EE126046A056AFD
:1008D00034EC28F0066EF3CF07F00750055C02E118
:1008E0000650045CD8B04CD0050E076E510E066E53
:1008F000800E086E0850E56E0750E56E0650E56EF6
:10090000A1EC20F0030EE12651C506F0076A000EA7
:100910000A6E2F0E096E840E086E000E0C6E600EAD
:100920000B6E800E0D6E0750E56E0650E56E0A5098
:10093000E56E0950E56E0850E56E0D50E56E0C5001
:10094000E56E0B50E56E18EC23F0080EE126000E64
:10095000076E600E066E800E086E0850E56E07503A
:10096000E56E0650E56E8DEC26F0030EE1260501DE
:100970005151E56EFDEC21F0E652044A052AA8D754
:10098000000E066E2F0E056E880E046E000E086EA9
:10099000600E076E800E096E0650E56E0550E56E1E
:1009A0000450E56E0950E56E0850E56E0750E56E9F
:1009B00018EC23F0060EE126000E056E600E046EA4
:1009C000800E066E0650E56E0550E56E0450E56E2D
:1009D0008DEC26F0030EE12634EC28F0046EF3CF04
:1009E00005F00450051027E06BEC28F0050E056EAD
:1009F000510E046E800E066E0650E56E0550E56ED3
:100A00000450E56EA1EC20F0046E030EE1260450C4
:100A10000FE005015151E56EFCEC28F0E652000EA6
:100A2000E56E040EE56EB6EC25F0E652E652DED732
:100A3000C3EC29F011D06BEC28F00D0EE56EFCEC48
:100A400028F0E652000EE56E040EE56EB6EC25F0D9
:100A5000E652E652C3EC29F002EC27F067EF07F00C
:100A600005EC2AF002EC27F0006A016A010EE56E3F
:100A7000900EE56EB6EC25F0E652E65234EC28F026
:100A8000026EF3CF03F00350015C02E10250005C00
:100A900012E202C000F003C001F0000EE56EC80EC5
:100AA000E56EB6EC25F0E652E65234EC28F0026E24
:100AB000F3CF03F0E8D705EC2AF0000E066E2F0EF8
:100AC000056E8C0E046E000E086E600E076E800EB2
:100AD000096E0650E56E0550E56E0450E56E09504E
:100AE000E56E0850E56E0750E56E18EC23F0060E33
:100AF000E126000E056E600E046E800E066E065036
:100B0000E56E0550E56E0450E56E8DEC26F0030EA3
:100B1000E126046A056A34EC28F0066EF3CF07F08C
:100B20000750055C02E10650045CD8B04CD0050EBD
:100B3000076E510E066E800E086E0850E56E075067
:100B4000E56E0650E56EA1EC20F0030EE12651C5DE
:100B500006F0076A000E0A6E2F0E096E840E086EEC
:100B6000000E0C6E600E0B6E800E0D6E0750E56E63
:100B70000650E56E0A50E56E0950E56E0850E56EC8
:100B80000D50E56E0C50E56E0B50E56E18EC23F041
:100B9000080EE126000E076E600E066E800E086ECF
:100BA0000850E56E0750E56E0650E56E8DEC26F0B8
:100BB000030EE12605015151E56EFDEC21F0E652F0
:100BC000044A052AA8D7000E066E2F0E056E880E61
:100BD000046E000E086E600E076E800E096E0650E1
:100BE000E56E0550E56E0450E56E0950E56E08505F
:100BF000E56E0750E56E18EC23F0060EE126000EB8
:100C0000056E600E046E800E066E0650E56E055091
:100C1000E56E0450E56E8DEC26F0030EE126E60E3F
:100C2000E56E1B0EE56EBBEC27F0E652E652050EB4
:100C3000056E510E046E800E066E0650E56E055070
:100C4000E56E0450E56EA1EC20F0046E030EE12683
:100C500004500FE005015151E56E85EC28F0E65295
:100C6000000EE56E0C0EE56EB6EC25F0E652E6528F
:100C7000DED7D9EC29F0E60EE56E1B0EE56E5BECD7
:100C800027F0E652E652006A016A050EE56EDC0EB8
:100C9000E56EB6EC25F0E652E65234EC28F0026E32
:100CA000F3CF03F00350015C02E10250005C12E25A
:100CB00002C000F003C001F0020EE56E580EE56EB2
:100CC000B6EC25F0E652E65234EC28F0026EF3CF93
:100CD00003F0E8D7CEEC29F0000E026E2F0E016E65
:100CE000800E006E000E046E600E036E800E056EA8
:100CF0000250E56E0150E56E0050E56E0550E56E60
:100D00000450E56E0350E56E18EC23F0060EE12664
:100D1000000E016E600E006E800E026E0250E56ED7
:100D20000150E56E0050E56E8DEC26F0030EE126D5
:100D3000006A016A34EC28F0026EF3CF03F003502E
:100D4000015C02E10250005CD8B04CD0050E036E8D
:100D5000510E026E800E046E0450E56E0350E56E77
:100D60000250E56EA1EC20F0030EE12651C502F021
:100D7000036A000E066E2F0E056E840E046E000EC2
:100D8000086E600E076E800E096E0350E56E02500D
:100D9000E56E0650E56E0550E56E0450E56E0950AF
:100DA000E56E0850E56E0750E56E18EC23F0080E6E
:100DB000E126000E036E600E026E800E046E04507B
:100DC000E56E0350E56E0250E56E8DEC26F0030EE5
:100DD000E12605015151E56EFDEC21F0E652004A95
:100DE000012AA8D7000E026E2F0E016E880E006E2B
:100DF000000E046E600E036E800E056E0250E56EEE
:100E00000150E56E0050E56E0550E56E0450E56E4C
:100E10000350E56E18EC23F0060EE126000E016E7D
:100E2000600E006E800E026E0250E56E0150E56E9F
:100E30000050E56E8DEC26F0030EE12634EC28F030
:100E4000006EF3CF01F00050011027E06BEC28F0AA
:100E5000050E016E510E006E800E026E0250E56EA0
:100E60000150E56E0050E56EA1EC20F0006E030E1F
:100E7000E12600500FE005015151E56EFCEC28F031
:100E8000E652000EE56E040EE56EB6EC25F0E65275
:100E9000E652DED7C3EC29F011D06BEC28F00D0E32
:100EA000E56EFCEC28F0E652000EE56E040EE56EF1
:100EB000B6EC25F0E652E652C3EC29F002EC27F03E
:100EC00006D005EC2AF0D6EC1BF002EC27F034EC4F
:100ED00028F0006EF3CF01F000500110D8B4ABEF52
:100EE00000F0050E016E510E006E800E026E025073
:100EF000E56E0150E56E0050E56EA1EC20F0030EAA
:100F0000E126E5D71200D9CFE5FFE1CFD9FF8282F4
:100F100000000000000000000000000000000000D1
:100F200000000000000000000000000000000000C1
:100F300000000000000000000000000000000000B1
:100F400000000000000000000000000000000000A1
:100F50000000000000000000000000000000000091
:100F60000000000000000000000000000000000081
:100F70000000000000000000000000000000000071
:100F80000000000000000000000000000000000061
:100F90000000000000000000000000000000000051
:100FA0000000000000000000000000000000000041
:100FB0000000000000000000000000000000000031
:100FC0000000000000000000000000000000000021
:100FD0000000000000000000000000000000000011
:100FE0000000000000000000000000000000000001
:100FF00000000000000000000000000000000000F1
:1010000000000000000000000000000000000000E0
:1010100000000000000000000000000000008292BC
:1010200000000000000000000000000000000000C0
:1010300000000000000000000000000000000000B0
:1010400000000000000000000000000000000000A0
:101050000000000000000000000000000000000090
:101060000000000000000000000000000000000080
:101070000000000000000000000000000000000070
:101080000000000000000000000000000000000060
:101090000000000000000000000000000000000050
:1010A0000000000000000000000000000000000040
:1010B0000000000000000000000000000000000030
:1010C0000000000000000000000000000000000020
:1010D0000000000000000000000000000000000010
:1010E0000000000000000000000000000000000000
:1010F00000000000000000000000000000000000F0
:1011000000000000000000000000000000000000DF
:1011100000000000000000000000000000000000CF
:1011200000000000000000000000000000008282BB
:1011300000000000000000000000000000000000AF
:10114000000000000000000000000000000000009F
:10115000000000000000000000000000000000008F
:10116000000000000000000000000000000000007F
:10117000000000000000000000000000000000006F
:10118000000000000000000000000000000000005F
:10119000000000000000000000000000000000004F
:1011A000000000000000000000000000000000003F
:1011B000000000000000000000000000000000002F
:1011C000000000000000000000000000000000001F
:1011D000000000000000000000000000000000000F
:1011E00000000000000000000000000000000000FF
:1011F00000000000000000000000000000000000EF
:1012000000000000000000000000000000000000DE
:1012100000000000000000000000000000000000CE
:1012200000000000000000000000000000000000BE
:10123000000000000000000000000000000082929A
:10124000000000000000000000000000000000009E
:10125000000000000000000000000000000000008E
:10126000000000000000000000000000000000007E
:10127000000000000000000000000000000000006E
:10128000000000000000000000000000000000005E
:10129000000000000000000000000000000000004E
:1012A000000000000000000000000000000000003E
:1012B000000000000000000000000000000000002E
:1012C000000000000000000000000000000000001E
:1012D000000000000000000000000000000000000E
:1012E00000000000000000000000000000000000FE
:1012F00000000000000000000000000000000000EE
:1013000000000000000000000000000000000000DD
:1013100000000000000000000000000000000000CD
:1013200000000000000000000000000000000000BD
:1013300000000000000000000000000000000000AD
:101340000000000000000000000000000000828299
:10135000000000000000000000000000000000008D
:10136000000000000000000000000000000000007D
:10137000000000000000000000000000000000006D
:10138000000000000000000000000000000000005D
:10139000000000000000000000000000000000004D
:1013A000000000000000000000000000000000003D
:1013B000000000000000000000000000000000002D
:1013C000000000000000000000000000000000001D
:1013D000000000000000000000000000000000000D
:1013E00000000000000000000000000000000000FD
:1013F00000000000000000000000000000000000ED
:1014000000000000000000000000000000000000DC
:1014100000000000000000000000000000000000CC
:1014200000000000000000000000000000000000BC
:1014300000000000000000000000000000000000AC
:10144000000000000000000000000000000000009C
:101450000000000000000000000000000000829278
:10146000000000000000000000000000000000007C
:10147000000000000000000000000000000000006C
:10148000000000000000000000000000000000005C
:10149000000000000000000000000000000000004C
:1014A000000000000000000000000000000000003C
:1014B000000000000000000000000000000000002C
:1014C000000000000000000000000000000000001C
:1014D000000000000000000000000000000000000C
:1014E00000000000000000000000000000000000FC
:1014F00000000000000000000000000000000000EC
:1015000000000000000000000000000000000000DB
:1015100000000000000000000000000000000000CB
:1015200000000000000000000000000000000000BB
:1015300000000000000000000000000000000000AB
:10154000000000000000000000000000000000009B
:10155000000000000000000000000000000000008B
:101560000000000000000000000000000000828277
:10157000000000000000000000000000000000006B
:10158000000000000000000000000000000000005B
:10159000000000000000000000000000000000004B
:1015A000000000000000000000000000000000003B
:1015B000000000000000000000000000000000002B
:1015C000000000000000000000000000000000001B
:1015D000000000000000000000000000000000000B
:1015E00000000000000000000000000000000000FB
:1015F00000000000000000000000000000000000EB
:1016000000000000000000000000000000000000DA
:1016100000000000000000000000000000000000CA
:1016200000000000000000000000000000000000BA
:1016300000000000000000000000000000000000AA
:10164000000000000000000000000000000000009A
:10165000000000000000000000000000000000008A
:10166000000000000000000000000000000000007A
:101670000000000000000000000000000000829256
:10168000000000000000000000000000000000005A
:10169000000000000000000000000000000000004A
:1016A000000000000000000000000000000000003A
:1016B000000000000000000000000000000000002A
:1016C000000000000000000000000000000000001A
:1016D000000000000000000000000000000000000A
:1016E00000000000000000000000000000000000FA
:1016F00000000000000000000000000000000000EA
:1017000000000000000000000000000000000000D9
:1017100000000000000000000000000000000000C9
:1017200000000000000000000000000000000000B9
:1017300000000000000000000000000000000000A9
:101740000000000000000000000000000000000099
:101750000000000000000000000000000000000089
:101760000000000000000000000000000000000079
:101770000000000000000000000000000000000069
:101780000000000000000000000000000000828255
:101790000000000000000000000000000000000049
:1017A0000000000000000000000000000000000039
:1017B0000000000000000000000000000000000029
:1017C0000000000000000000000000000000000019
:1017D0000000000000000000000000000000000009
:1017E00000000000000000000000000000000000F9
:1017F00000000000000000000000000000000000E9
:1018000000000000000000000000000000000000D8
:1018100000000000000000000000000000000000C8
:1018200000000000000000000000000000000000B8
:1018300000000000000000000000000000000000A8
:101840000000000000000000000000000000000098
:101850000000000000000000000000000000000088
:101860000000000000000000000000000000000078
:101870000000000000000000000000000000000068
:101880000000000000000000000000000000000058
:101890000000000000000000000000000000829234
:1018A0000000000000000000000000000000000038
:1018B0000000000000000000000000000000000028
:1018C0000000000000000000000000000000000018
:1018D0000000000000000000000000000000000008
:1018E00000000000000000000000000000000000F8
:1018F00000000000000000000000000000000000E8
:1019000000000000000000000000000000000000D7
:1019100000000000000000000000000000000000C7
:1019200000000000000000000000000000000000B7
:1019300000000000000000000000000000000000A7
:101940000000000000000000000000000000000097
:101950000000000000000000000000000000000087
:101960000000000000000000000000000000000077
:101970000000000000000000000000000000000067
:101980000000000000000000000000000000000057
:101990000000000000000000000000000000000047
:1019A0000000000000000000000000000000828233
:1019B0000000000000000000000000000000000027
:1019C0000000000000000000000000000000000017
:1019D0000000000000000000000000000000000007
:1019E00000000000000000000000000000000000F7
:1019F00000000000000000000000000000000000E7
:101A000000000000000000000000000000000000D6
:101A100000000000000000000000000000000000C6
:101A200000000000000000000000000000000000B6
:101A300000000000000000000000000000000000A6
:101A40000000000000000000000000000000000096
:101A50000000000000000000000000000000000086
:101A60000000000000000000000000000000000076
:101A70000000000000000000000000000000000066
:101A80000000000000000000000000000000000056
:101A90000000000000000000000000000000000046
:101AA0000000000000000000000000000000000036
:101AB0000000000000000000000000000000829212
:101AC000E4CFD9FF1200D9CFE5FFE1CFD9FF828261
:101AD0000000000000000000000000000000000006
:101AE00000000000000000000000000000000000F6
:101AF00000000000000000000000000000000000E6
:101B000000000000000000000000000000000000D5
:101B100000000000000000000000000000000000C5
:101B200000000000000000000000000000000000B5
:101B300000000000000000000000000000000000A5
:101B40000000000000000000000000000000000095
:101B50000000000000000000000000000000000085
:101B60000000000000000000000000000000000075
:101B70000000000000000000000000000000000065
:101B80000000000000000000000000000000000055
:101B90000000000000000000000000000000000045
:101BA0000000000000000000000000000000000035
:101BB0000000000000000000000000000000000025
:101BC0000000000000000000000000000000000015
:101BD0000000000000000000000000000000000005
:101BE00000000000000000000000000000000000F5
:101BF00000000000000000000000000000000000E5
:101C000000000000000000000000000000000000D4
:101C100000000000000000000000000000000000C4
:101C200000000000000000000000000000000000B4
:101C300000000000000000000000000000000000A4
:101C40000000000000000000000000000000000094
:101C50000000000000000000000000000000000084
:101C60000000000000000000829200000000000060
:101C70000000000000000000000000000000000064
:101C80000000000000000000000000000000000054
:101C90000000000000000000000000000000000044
:101CA0000000000000000000000000000000000034
:101CB0000000000000000000000000000000000024
:101CC0000000000000000000000000000000000014
:101CD0000000000000000000000000000000000004
:101CE00000000000000000000000000000000000F4
:101CF00000000000000000000000000000000000E4
:101D000000000000000000000000000000000000D3
:101D100000000000000000000000000000000000C3
:101D200000000000000000000000000000000000B3
:101D300000000000000000000000000000000000A3
:101D40000000000000000000000000000000000093
:101D50000000000000000000000000000000000083
:101D60000000000000000000000000000000000073
:101D70000000000000000000000000000000000063
:101D80000000000000000000000000000000000053
:101D90000000000000000000000000000000000043
:101DA0000000000000000000000000000000000033
:101DB0000000000000000000000000000000000023
:101DC0000000000000000000000000000000000013
:101DD0000000000000000000000000000000000003
:101DE00000000000000000000000000000000000F3
:101DF00000000000000000000000000000000000E3
:101E000000008282000000000000000000000000CE
:101E100000000000000000000000000000000000C2
:101E200000000000000000000000000000000000B2
:101E300000000000000000000000000000000000A2
:101E40000000000000000000000000000000000092
:101E50000000000000000000000000000000000082
:101E60000000000000000000000000000000000072
:101E70000000000000000000000000000000000062
:101E80000000000000000000000000000000000052
:101E90000000000000000000000000000000000042
:101EA0000000000000000000000000000000000032
:101EB0000000000000000000000000000000000022
:101EC0000000000000000000000000000000000012
:101ED0000000000000000000000000000000000002
:101EE00000000000000000000000000000000000F2
:101EF00000000000000000000000000000000000E2
:101F000000000000000000000000000000000000D1
:101F100000000000000000000000000000000000C1
:101F200000000000000000000000000000000000B1
:101F300000000000000000000000000000000000A1
:101F40000000000000000000000000000000000091
:101F50000000000000000000000000000000000081
:101F60000000000000000000000000000000000071
:101F70000000000000000000000000000000000061
:101F80000000000000000000000000000000000051
:101F9000000000000000000000000000829200002D
:101FA0000000000000000000000000000000000031
:101FB0000000000000000000000000000000000021
:101FC0000000000000000000000000000000000011
:101FD0000000000000000000000000000000000001
:101FE00000000000000000000000000000000000F1
:101FF00000000000000000000000000000000000E1
:1020000000000000000000000000000000000000D0
:1020100000000000000000000000000000000000C0
:1020200000000000000000000000000000000000B0
:1020300000000000000000000000000000000000A0
:102040000000000000000000000000000000000090
:102050000000000000000000000000000000000080
:102060000000000000000000000000000000000070
:102070000000000000000000000000000000000060
:102080000000000000000000000000000000000050
:102090000000000000000000000000000000000040
:1020A0000000000000000000000000000000000030
:1020B0000000000000000000000000000000000020
:1020C0000000000000000000000000000000000010
:1020D0000000000000000000000000000000000000
:1020E00000000000000000000000000000000000F0
:1020F00000000000000000000000000000000000E0
:1021000000000000000000000000000000000000CF
:1021100000000000000000000000000000000000BF
:1021200000000000000000000000000000000000AF
:10213000000000000000828200000000000000009B
:10214000000000000000000000000000000000008F
:10215000000000000000000000000000000000007F
:10216000000000000000000000000000000000006F
:10217000000000000000000000000000000000005F
:10218000000000000000000000000000000000004F
:10219000000000000000000000000000000000003F
:1021A000000000000000000000000000000000002F
:1021B000000000000000000000000000000000001F
:1021C000000000000000000000000000000000000F
:1021D00000000000000000000000000000000000FF
:1021E00000000000000000000000000000000000EF
:1021F00000000000000000000000000000000000DF
:1022000000000000000000000000000000000000CE
:1022100000000000000000000000000000000000BE
:1022200000000000000000000000000000000000AE
:10223000000000000000000000000000000000009E
:10224000000000000000000000000000000000008E
:10225000000000000000000000000000000000007E
:10226000000000000000000000000000000000006E
:10227000000000000000000000000000000000005E
:10228000000000000000000000000000000000004E
:10229000000000000000000000000000000000003E
:1022A000000000000000000000000000000000002E
:1022B000000000000000000000000000000000001E
:1022C000000000000000000000000000000000000E
:1022D00082920000000000000000000000000000EA
:1022E00000000000000000000000000000000000EE
:1022F00000000000000000000000000000000000DE
:1023000000000000000000000000000000000000CD
:1023100000000000000000000000000000000000BD
:1023200000000000000000000000000000000000AD
:10233000000000000000000000000000000000009D
:10234000000000000000000000000000000000008D
:10235000000000000000000000000000000000007D
:10236000000000000000000000000000000000006D
:10237000000000000000000000000000000000005D
:10238000000000000000000000000000000000004D
:10239000000000000000000000000000000000003D
:1023A000000000000000000000000000000000002D
:1023B000000000000000000000000000000000001D
:1023C000000000000000000000000000000000000D
:1023D00000000000000000000000000000000000FD
:1023E00000000000000000000000000000000000ED
:1023F00000000000000000000000000000000000DD
:1024000000000000000000000000000000000000CC
:1024100000000000000000000000000000000000BC
:1024200000000000000000000000000000000000AC
:10243000000000000000000000000000000000009C
:10244000000000000000000000000000000000008C
:10245000000000000000000000000000000000007C
:102460000000000000000000000082820000000068
:10247000000000000000000000000000000000005C
:10248000000000000000000000000000000000004C
:10249000000000000000000000000000000000003C
:1024A000000000000000000000000000000000002C
:1024B000000000000000000000000000000000001C
:1024C000000000000000000000000000000000000C
:1024D00000000000000000000000000000000000FC
:1024E00000000000000000000000000000000000EC
:1024F00000000000000000000000000000000000DC
:1025000000000000000000000000000000000000CB
:1025100000000000000000000000000000000000BB
:1025200000000000000000000000000000000000AB
:10253000000000000000000000000000000000009B
:10254000000000000000000000000000000000008B
:10255000000000000000000000000000000000007B
:10256000000000000000000000000000000000006B
:10257000000000000000000000000000000000005B
:10258000000000000000000000000000000000004B
:10259000000000000000000000000000000000003B
:1025A000000000000000000000000000000000002B
:1025B000000000000000000000000000000000001B
:1025C000000000000000000000000000000000000B
:1025D00000000000000000000000000000000000FB
:1025E00000000000000000000000000000000000EB
:1025F00000000000000000000000000000000000DB
:10260000000000008292E4CFD9FF1200D8CFE5FF8E
:10261000E0CFE5FFE56EF3CFE5FFF4CFE5FFE9CFCF
:10262000E5FFEACFE5FFFACFE5FFFBCFE5FFD9CF26
:10263000E5FFE1CFD9FF00C0E5FF01C0E5FF02C023
:10264000E5FF03C0E5FF04C0E5FF05C0E5FFF2A21A
:10265000A1D1F2A89FD1D6CF00F0016AD7CF02F066
:10266000036A0250056E046A045000100501476FAA
:1026700005500110486F05014A51006E016A005073
:10268000D76E4951D66E05015251010A0BE0050182
:102690005251020A01E11DD105015251040A01E122
:1026A00046D177D1640EE56E65EC29F0E65224C57B
:1026B00000F00050016E015008E00050020A0CE0EA
:1026C0000050040A01E13BD064D1D58E010E050112
:1026D000266F020E246F5DD1050149518F0F006EE8
:1026E000020E4A21016E05014851015C02E1475189
:1026F000005C1FE2050149511F0F006E040E4A21C4
:10270000016E01500501485D02E10050475D11E294
:1027100026C500F0020E005C05E2002A005005010B
:10272000266F37D10501276B286B296B040E246FA8
:1027300030D1010E0501266F020E246F2AD10D0E35
:102740000501295DD8B025D1050149518F0F006ED3
:10275000020E4A21016E05014851015C02E1475118
:10276000005C0EE2050149511F0F006E040E4A2164
:10277000016E01500501485D02E10050475D1CE318
:10278000050149513D0F006E090E4A21016E0501F8
:102790004851015C02E14751005C35E205014951B5
:1027A000CD0F006E0A0E4A21016E01500501485DF1
:1027B00002E10050475D27E227C500F028C501F07F
:1027C00000A00BD00050026E02260134036E0250AE
:1027D0000501276F0350286F0FD00050026E0226AC
:1027E0000134036E02500501276F0350286F0280E9
:1027F0000250276F0350286F29C500F0002A0050AF
:102800000501296F48D005014951E60F006E050EFC
:102810004A21016E05014851015C02E14751005C0B
:1028200035E205014951760F006E070E4A21016E0F
:1028300001500501485D02E10050475D27E227C5D0
:1028400000F028C501F000A010D00050026E022652
:102850000134036E02500501276F0350286F028078
:102860000250276F0350286F0AD00050026E0226D4
:102870000134036E02500501276F0350286F29C5EC
:1028800000F0002A00500501296F05D0010E050156
:10289000266F020E246F050129510C0A01E079D040
:1028A00005012851E56E2751E56EF5EC1DF0006E2F
:1028B000E652E65200500AE005012751006E016A17
:1028C0000050E56EFDEC21F0E65281880501246B95
:1028D00060D005011D51020A01E05BD0050149519C
:1028E000FF08006EFF0E4A55016ED890013200328B
:1028F0000050495D006E01504A59016E0150006E52
:10290000016A0050D76E4951006E4951FF08016EAF
:10291000FF0E4A55026ED890023201320150005C1F
:10292000D66EF298D58E040E05011D6F32D00501CA
:102930001D51020A2EE105014951FF08006EFF0EEC
:102940004A55016ED890013200320050495D006E48
:1029500001504A59016E0150006E016A0050D76E55
:102960004951006E4951FF08016EFF0E4A55026E33
:10297000D890023201320150005CD66EF298D58EAA
:102980007F0E05011F15006E00501F6F226B040E95
:102990001D6FF292F2A4ECEF16F0F2AAECEF16F033
:1029A00005014A51006E016A0050D76E4951D66E3A
:1029B000010E0501525DD8A0EBEF16F0080E525D36
:1029C000D8B0EBEF16F05205006EFA6AFB6A0034DD
:1029D000FA36E834FA36FC0BE80FE56E290EFA22D7
:1029E000000EFB22E450F96E02EF15F051EF15F0E6
:1029F00008EF15F0F9EF15F08FEF15F053EF16F023
:102A000096EF16F0D59E0501246B0300EBEF16F050
:102A10001DC500F00050016E01500AE00050030A8D
:102A200011E000500A0A33E000500B0A35E0D3D120
:102A300005012051080A01E0CED18182030E050173
:102A40001D6FC9D1010E0501205D1CE3010E1F158C
:102A5000006E0050D880E866D890006A00360050BA
:102A6000010BE844F46E8150FD0BF410816E1F41A0
:102A70007F0B006E00501F6F20C500F00006005055
:102A8000206FA9D181920A0E05011D6FA4D18192F8
:102A90000B0E05011D6F9FD1819205011D6BD59E07
:102AA0009AD11DC500F00050040A07E00050080A42
:102AB00023E00050090A24E08ED120C500F0002A4E
:102AC00000500501206F81A006D01F417F0B006ED2
:102AD00000501F6F09D005011F417F0B006E005091
:102AE0001F6F008E00501F6F080E0501205DD8A0DB
:102AF00072D1080E1D6F6FD1090E05011D6F6BD1CC
:102B000005011F51E56EFDEC21F0E65205011F6B3A
:102B1000206B020E1D6FD59EF292F2885CD11DC50E
:102B200000F00050016E01500CE00050030A18E064
:102B30000050060A01E153D000500A0A01E154D0C6
:102B40004AD105012051070A01E045D18182010ED9
:102B500005011F15006E0050216F030E1D6F3BD144
:102B6000010E0501205D26E3010E1F15006E0050C9
:102B7000D880E866D890006A00360050010BE8441F
:102B8000F46E8150FD0BF410816E1F51020BE84072
:102B9000006E2151016E0150001A0050216F1F413B
:102BA0007F0B006E00501F6F20C500F00006005024
:102BB000206F11D1010E05012115006E0050D88043
:102BC000E866D890006A00360050010BE844F46EC5
:102BD0008150FD0BF410816E060E1D6FFCD08192AA
:102BE0000A0E05011D6FF7D0819205011D6BD59E60
:102BF000F2D01DC500F00050040A07E00050070A9B
:102C00002CE00050080A35E0E6D020C500F0002A8C
:102C100000500501206F81A00AD022C500F00050AD
:102C2000226F1F417F0B006E00501F6F0ED0010EF0
:102C300005012219006E0050226F1F417F0B006EAC
:102C400000501F6F008C00501F6F070E0501205DA4
:102C5000D8A0C1D0070E1D6FBED081A002D0006ADF
:102C600002D0010E006E00500501216F080E1D6F8D
:102C7000B2D005012251211907E105011F51E56E6E
:102C8000FDEC21F0E65206D005011F51E56EFDEC8A
:102C900021F0E65205011F6B206B020E1D6FD59EC1
:102CA000F292F28898D000C500F00050040A04E0C7
:102CB0000050080A2FE08FD00DC500F0002A005008
:102CC00005010D6F090E005C21E201C500F002C58F
:102CD00001F0010E015C02E1550E005C0DE3010EF6
:102CE000015C02E1DC0E005C07E205010C417F0B98
:102CF000006E00500C6F6FD005010C417F0B006E11
:102D000000500C6F008E00500C6F65D0080E05014E
:102D1000006F61D005010C51E56EFDEC21F0E6522B
:102D200005010C6B020E006FF29A55D000C500F041
:102D30000050016E01500FE00050010A15E00050F4
:102D4000030A19E00050050A01E139D000500A0ACF
:102D500001E13CD040D005010D51080A03E1010E0C
:102D60000501006F819837D063EC0DF0030E05016B
:102D7000006F818830D00DC500F00004016E015055
:102D800005010D6F005015E0800E006E0D5105E03D
:102D9000E86CD8900032010FFDE305010C510016DC
:102DA000005004E083EC07F0819803D063EC0DF051
:102DB000818805010D510FE1050E006F0CD083ECE9
:102DC00007F00A0E0501006F819805D083EC07F02B
:102DD0000501006B8198F294A1AC77D0A0AC75D0BE
:102DE000B4AC71D0D6CF00F0016AD7CF02F0036A3D
:102DF0000250056E046A045000100501476F05502B
:102E00000110486F818805014B510501475D006E37
:102E100005014C5105014859016E00500501016F33
:102E20000150026F47C54BF548C54CF501C500F090
:102E300002C501F0010E015C02E1550E005C2DE3BC
:102E4000010E015C02E1DC0E005C27E20501055188
:102E50000026065101220050056F0150066F0051F7
:102E6000020A32E1030E0501065D02E1200E055D56
:102E70002BE305014A51006E016A0050D76E49519B
:102E8000D66E0501056B066B076B086B0D6B0C6B43
:102E9000040E006FF294F28A17D005010051020A65
:102EA00006E10501056B066B076B086B0DD005018C
:102EB00001510725006E02510821016E0050076F75
:102EC0000150086F01D08198A19CE4CF05F0E4CFB8
:102ED00004F0E4CF03F0E4CF02F0E4CF01F0E4CF5C
:102EE00000F0E4CFD9FFE4CFFBFFE4CFFAFFE4CF5B
:102EF000EAFFE4CFE9FFE4CFF4FFE4CFF3FFE450CF
:102F0000E4CFE0FFE4CFD8FF100050726F63657329
:102F1000736F723A20706963313866323535300A22
:102F20000D0050726F636573736F723A207069633E
:102F3000313866323535330A0D0050726F63657370
:102F4000736F723A20756E737570706F727465640A
:102F50002C206465766963652069643A20307825A1
:102F60003034780A0D000A0D707265737320707228
:102F7000696E74206F6E20746573746F0A0D0000A3
:102F80003C2D2000256420000A0D00002D3E20006D
:102F9000426174746572793A2025646D560A0D0099
:102FA000D9CFE5FFE1CFD9FF00C0E5FF01C0E5FFC4
:102FB00002C0E5FF03C0E5FF04C0E5FF05C0E5FF73
:102FC00006C0E5FF07C0E5FF08C0E5FF09C0E5FF53
:102FD0000AC0E5FF0BC0E5FF0CC0E5FF0DC0E5FF33
:102FE0000EC0E5FF0FC0E5FF10C0E5FF11C0E5FF13
:102FF00012C0E5FF13C0E5FF14C0E5FF15C0E5FFF3
:1030000016C0E5FF17C0E5FF18C0E5FF19C0E5FFD2
:103010001AC0E5FF1BC0E5FF1CC0E5FF1DC0E5FFB2
:103020001EC0E5FF020EDBCF00F0030EDBCF01F088
:10303000040EDBCF02F0050EDBCF03F0060EDBCF74
:1030400004F0070EDBCF05F0080EDBCF06F0090E0B
:10305000DBCF07F00A0EDBCF08F0096A0A6A02C06C
:103060000DF00D50800A0DE102500501406F015036
:103070003F6F00503E6F050E016E3E0E006E800EDB
:10308000026E03C0E9FF04C0F3FF055077EC29F09E
:103090000B6E0B50D8B48CEF1BF00B50250A02E0DE
:1030A00073EF1BF00C6A0D6A0E6A0F6A106A0A0E43
:1030B000116E126A136A146A200E156E1668176A6A
:1030C0002B0E186E032A02E3044A052A03C0E9FF07
:1030D00004C0F3FF055077EC29F0196E250A13E1BF
:1030E0001950E56E0250E56E0150E56E0050E56E38
:1030F000A2EC23F0040EE126094A0A2A032A02E37D
:10310000044A052ABED71950300A06E1300E156E62
:10311000032A02E3044A052A03C0E9FF04C0F3FFBF
:10312000055077EC29F02D0A06E1010E146E032AF2
:1031300002E3044A052A03C0E9FF04C0F3FF055077
:1031400077EC29F0200A08E1010E176E200E186EA8
:10315000032A02E3044A052A03C0E9FF04C0F3FF7F
:10316000055077EC29F02B0A06E1010E176E032AB1
:1031700002E3044A052A03C0E9FF04C0F3FF055037
:1031800077EC29F0196E800F4F0F2DE31950800F47
:10319000460F29E203C019F004C01AF005C01BF065
:1031A00019C0E9FF1AC0F3FF1B5077EC29F01C6E21
:1031B000800F500F12E31C50800F460F0EE2135089
:1031C0000A0DF3CF1DF01D501C26D00E1C24136ECB
:1031D000192A02E31A4A1B2AE3D719C003F01AC0BE
:1031E00004F01BC005F003C0E9FF04C0F3FF055065
:1031F00077EC29F02E0A2EE1032A02E3044A052A7D
:10320000166A03C019F004C01AF005C01BF019C0FB
:10321000E9FF1AC0F3FF1B5077EC29F01C6E800FFA
:10322000500F12E31C50800F460F0EE216500A0D8D
:10323000F3CF1DF01D501C26D00E1C24166E192A2B
:1032400002E31A4A1B2AE3D719C003F01AC004F09C
:103250001BC005F003C0E9FF04C0F3FF055077EC85
:1032600029F0196E6C0A07E1010E0C6E032A02E3C5
:10327000044A052A09D01950680A06E1010E0E6EAB
:10328000032A02E3044A052A03C0E9FF04C0F3FF4E
:10329000055077EC29F0750A06E1010E106E032A3D
:1032A00002E3044A052A03C0E9FF04C0F3FF055006
:1032B00077EC29F0196E730A05E1010E0D6E200EF0
:1032C000156E3FD01950780A03E1100E116E39D0F7
:1032D0001950580A05E1100E116E010E126E31D010
:1032E0001950630A02E1116A2CD019506F0A03E1E8
:1032F000080E116E26D01950660A03E1010E0F6EFA
:1033000020D01950640A1DE01950690A1AE01050C3
:1033100005E0FF0E03260422052213D01950E56EA6
:103320000250E56E0150E56E0050E56EA2EC23F010
:10333000040EE126094A0A2A032A02E3044A052A5E
:10334000A0D60D5021E00650030F0D6E000E072091
:10335000196E000E08201A6E0DC006F019C007F095
:103360001AC008F0FD0E0D26FF0E19221A220DC0FC
:10337000E9FF19C0F3FF1A5050EC28F00D6EF3CF9F
:1033800019F0F4CF1AF000D10F500DE0000E1A6EB4
:10339000370E196EA00E0D6E040E0626000E0722C3
:1033A00008221668F1D016680C5023E00650040F6E
:1033B0000C6E000E07200F6E000E08201B6E0CC056
:1033C00006F00FC007F01BC008F0FC0E0C26FF0E25
:1033D0000F221B220CC0E9FF0FC0F3FF1B509BEC18
:1033E00027F00C6EF3CF0FF0F4CF1BF0E9CF1CF0F9
:1033F0006AD00E5032E00650020F0E6E000E07200B
:103400001D6E000E08201E6E0EC006F01DC007F0D7
:103410001EC008F0FE0E0E26FF0E1D221E220EC03C
:10342000E9FF1DC0F3FF1E5012EC29F00E6E0EC016
:103430000CF0E86A0EBEFF0E0F6E1B6E1C6E115074
:103440000A0A03E11050D8B43ED00C500E6E0EC0E4
:103450000CF00F6A1B6A1C6A36D00650020F0E6E03
:10346000000E07201D6E000E08201E6E0EC006F016
:103470001DC007F01EC008F0FE0E0E26FF0E1D2216
:103480001E220EC0E9FF1DC0F3FF1E5012EC29F0F2
:103490000E6EF3CF1DF00EC00CF01DC00FF0E86AE9
:1034A0001DBEFF0E1B6E1C6E11500A0A02E1105069
:1034B0000AE00C500E6E0F501D6E0EC00CF01DC0B9
:1034C0000FF01B6A1C6A050E196E110E0D6E800E30
:1034D0001A6E1150D8B440D0105013E01150E56E60
:1034E000050EE56E110EE56E1C50E56E1B50E56E87
:1034F0000F50E56E0C50E56EF5EC1EF0070EE12660
:1035000012D01150E56E050EE56E110EE56E1C50E1
:10351000E56E1B50E56E0F50E56E0C50E56EF1EC5C
:1035200024F0070EE12617502FE00DC0E9FF19C067
:10353000F3FF1A5077EC29F02D0A26E0FF0E0D2636
:1035400019221A2218C0E5FF0DC0E9FF19C0F3FFC8
:103550001A50FAEC29F018D00CC0E5FF0DC0E9FFB5
:1035600019C0F3FF1A50FAEC29F00D50010F0C6E40
:10357000000E19200E6E000E1A20E56A0CC0E9FF3D
:103580000EC0F3FFFAEC29F00DC00CF019C00EF0DC
:103590001AC00FF013C010F0105010E00CC0E9FF7B
:1035A0000EC0F3FF0F5077EC29F0176E175006E0AE
:1035B0000C2A02E30E4A0F2A1006EED710C013F0B1
:1035C00014501EE109C00CF00AC00EF010C00FF03C
:1035D0000F5010E01550E56E0250E56E0150E56E9B
:1035E0000050E56EA2EC23F0040EE1260C4A0E2AF0
:1035F0000F06EED70CC009F00EC00AF00FC013F092
:1036000016C00CF00DC00DF019C00EF01AC00FF06E
:1036100009C010F00AC015F00DC0E9FF0EC0F3FF9D
:103620000F5077EC29F0166E1650D8B43ED00CC06F
:1036300016F0176A161E171E1650171005E00CC05C
:1036400016F00C06165031E00DC0E9FF0EC0F3FF76
:103650000F5077EC29F0116E125010E01150E56E0A
:10366000E5EC28F0166EE652165004E01150166E86
:10367000169A02D011C016F016C011F01150E56E66
:103680000250E56E0150E56E0050E56EA2EC23F0AD
:10369000040EE1260D2A02E30E4A0F2A104A152ACB
:1036A0001350D8B4B9D71306B7D710C009F015C056
:1036B0000AF014502BE010C00CF015C00DF013C030
:1036C0000EF00E501FE0200EE56E0250E56E015028
:1036D000E56E0050E56EA2EC23F0040EE1260C4AE4
:1036E0000D2A0E06EED70B50E56E0250E56E015026
:1036F000E56E0050E56EA2EC23F0040EE126094AC7
:103700000A2A04D00CC009F00DC00AF0032A02E313
:10371000044A052A41EF18F00AC0F3FF0950E4CF2C
:103720001EF0E4CF1DF0E4CF1CF0E4CF1BF0E4CF9B
:103730001AF0E4CF19F0E4CF18F0E4CF17F0E4CF9B
:1037400016F0E4CF15F0E4CF14F0E4CF13F0E4CF9B
:1037500012F0E4CF11F0E4CF10F0E4CF0FF0E4CF9B
:103760000EF0E4CF0DF0E4CF0CF0E4CF0BF0E4CF9B
:103770000AF0E4CF09F0E4CF08F0E4CF07F0E4CF9B
:1037800006F0E4CF05F0E4CF04F0E4CF03F0E4CF9B
:1037900002F0E4CF01F0E4CF00F0E4CFD9FF120053
:1037A0003C4E4F20464C4F41543E0000D9CFE5FFE0
:1037B000E1CFD9FF00C0E5FF01C0E5FF02C0E5FF92
:1037C00003C0E5FF04C0E5FF05C0E5FF06C0E5FF57
:1037D00007C0E5FF800EE56E0A0EE56E060EE56E8B
:1037E000040EE56E4FEC26F0040EE126040EE56EA5
:1037F00017EC28F0E6520AEC00F03BEC2AF0006EE1
:103800000050FBE1C9EC26F0006EF3CF01F0005050
:10381000400A03E10150120A01E041D033EC2AF0E2
:10382000026EF3CF03F0E86A03BEFF0E046E056E6E
:103830000550E56E0450E56E0350E56E0250E56EEE
:10384000000EE56E0C0EE56EB50EE56EE80EE56E4B
:10385000EBEC1CF0026EF3CF03F0F4CF04F0E9CFF1
:1038600005F0080EE126000EE56E010EE56E6D0E08
:10387000E56EA00EE56E0550E56E0450E56E035052
:10388000E56E0250E56E8CEC22F0026EF3CF03F091
:10389000F4CF04F0E9CF05F0080EE12654D0005033
:1038A000400A03E101502A0A01E04BD033EC2AF030
:1038B000006EF3CF01F001340132003201340132E5
:1038C0000032E86A01BEFF0E046E056E0550E56E1B
:1038D0000450E56E0150E56E0050E56E000EE56E99
:1038E0000C0EE56EB50EE56EE80EE56EEBEC1CF029
:1038F000006EF3CF01F0F4CF04F0E9CF05F0080E2D
:10390000E126000EE56E010EE56E6D0EE56EA00E71
:10391000E56E0550E56E0450E56E0150E56E005011
:10392000E56E8CEC22F0006EF3CF01F0F4CF04F0E2
:10393000E9CF05F0080EE1260050026E0150036E3B
:1039400002D0026A036A000E046E2F0E016E900E02
:10395000006E000E066E600E056E800E076E035040
:10396000E56E0250E56E0450E56E0150E56E0050C4
:10397000E56E0750E56E0650E56E0550E56E18ECF5
:1039800023F0080EE126000E016E600E006E800E20
:10399000046E0450E56E0150E56E0050E56E8DEC4E
:1039A00026F0030EE12646EC2AF003C0F3FF025096
:1039B000E4CF07F0E4CF06F0E4CF05F0E4CF04F065
:1039C000E4CF03F0E4CF02F0E4CF01F0E4CF00F065
:1039D000E4CFD9FF1200D9CFE5FFE1CFD9FF00C076
:1039E000E5FF01C0E5FF02C0E5FF03C0E5FF04C03D
:1039F000E5FF05C0E5FF06C0E5FF07C0E5FF020ED5
:103A0000DBCF00F0030EDBCF01F0040EDBCF02F0C2
:103A1000050EDBCF03F0060EDBCF04F0070EDBCF85
:103A200005F0080EDBCF06F0090EDBCF07F00050E3
:103A300005012A6F01502B6F02502C6F03502D6F20
:103A4000045005012E6F05502F6F0650306F075040
:103A5000316F05012A5105013003F4CF01F0F3CF96
:103A600000F000500501346F0150356F05012A51F7
:103A700005012E03F4CF01F0F3CF00F00050050153
:103A8000326F0150336F05012D5105012E03F3CF25
:103A900000F00501355100260050356F05012C510D
:103AA00005012F03F3CF00F005013551002600502A
:103AB000356F05012C5105012E03F4CF01F0F3CF32
:103AC00000F0050134510026355101220050346FB9
:103AD0000150356F05012B5105012F03F4CF01F083
:103AE000F3CF00F00501345100263551012200507A
:103AF000346F0150356F05012B5105013003F3CFB1
:103B000000F000500501396F05012B5105012E030E
:103B1000F4CF01F0F3CF00F000500501376F0150F2
:103B2000386F05012A5105013103F3CF00F0005031
:103B300005013D6F05012A5105012F03F4CF01F066
:103B4000F3CF00F0005005013B6F01503C6F0501C1
:103B5000366B05013A6B0501365105013225006EC1
:103B60000501375105013321016E05013851050169
:103B70003421026E0501395105013521036E0050D3
:103B8000326F0150336F0250346F0350356F0501AF
:103B90003A5105013225006E05013B5105013321E3
:103BA000016E05013C5105013421026E05013D51B4
:103BB00005013521036E03C0E9FF02C0F4FF01C017
:103BC000F3FF0050E4CF07F0E4CF06F0E4CF05F0B8
:103BD000E4CF04F0E4CF03F0E4CF02F0E4CF01F04F
:103BE000E4CF00F0E4CFD9FF1200D9CFE5FFE1CF59
:103BF000D9FF00C0E5FF01C0E5FF02C0E5FF03C03B
:103C0000E5FF04C0E5FF05C0E5FF06C0E5FF07C00E
:103C1000E5FF08C0E5FF020EDBCF00F0030EDBCFAF
:103C200001F0026A780E0014036E046A056A010E40
:103C3000066E000E076E055006E0E86CD89006365A
:103C40000736010FFCE30350061604500716065012
:103C500005E1075003E1066A062A01D0066A06500C
:103C6000D880E866D890066A06360250076E06507D
:103C70000718026E052A080E055CD9E30244FE0B04
:103C8000036E026AE60E0014046E056A066A010EEF
:103C9000076E000E086E065006E0E86CD8900736F6
:103CA0000836010FFCE304500716055008160750AC
:103CB00005E1085003E1076A072A01D0076A0750A7
:103CC000D880E866D890076A07360250086E075019
:103CD0000818026E062A080E065CD9E30250031289
:103CE000D8900336026AD50E0014046E056A066A7F
:103CF000010E076E000E086E065006E0E86CD890C4
:103D000007360836010FFCE3045007160550081665
:103D1000075005E1085003E1076A072A01D0076A46
:103D20000750D880E866D890076A07360250086EB8
:103D300007500818026E062A080E065CD9E30250E6
:103D40000312D8900336026A8B0E0014046E056AC3
:103D5000066A010E076E000E086E065006E0E86C5B
:103D6000D89007360836010FFCE3045007160550BB
:103D70000816075005E1085003E1076A072A01D039
:103D8000076A0750D880E866D890076A073602505D
:103D9000086E07500818026E062A080E065CD9E362
:103DA000025003120150006E016A026A00500318AB
:103DB00003E10150021801E002D0010E01D0E86ACF
:103DC000E4CF08F0E4CF07F0E4CF06F0E4CF05F04D
:103DD000E4CF04F0E4CF03F0E4CF02F0E4CF01F04D
:103DE000E4CF00F0E4CFD9FF1200D9CFE5FFE1CF57
:103DF000D9FF00C0E5FF01C0E5FF02C0E5FF03C039
:103E0000E5FF04C0E5FF05C0E5FF06C0E5FF07C00C
:103E1000E5FF08C0E5FF09C0E5FF0AC0E5FF0BC0EC
:103E2000E5FF0CC0E5FF0DC0E5FF0EC0E5FF0FC0CC
:103E3000E5FF020EDBCF00F0030EDBCF01F0040E36
:103E4000DBCF02F0050EDBCF03F0060EDBCF04F074
:103E5000070EDBCF05F0080EDBCF06F0200E076E55
:103E6000086A06C009F00A6A0B6A0C6AE56AE56A24
